:020000040800F2
:1000000000040020973E0008591B00085B1B0008F5
:10001000831B0008871B00088B1B000800000000E2
:100020000000000000000000000000008F1B00081E
:10003000911B000800000000931B0008951B00089E
:10004000B73E0008B73E0008B73E0008B73E0008BC
:10005000B73E0008B73E0008B73E0008B73E0008AC
:10006000B73E0008B73E0008B73E0008B73E00089C
:10007000B73E0008B73E0008B73E0008B73E00088C
:10008000B73E0008B73E0008B73E0008B73E00087C
:10009000B73E0008B73E0008B73E0008B73E00086C
:1000A000B73E0008B73E0008B73E0008B73E00085C
:1000B000B73E0008B73E0008571B0008B73E0008CF
:1000C000B73E0008B73E0008B73E0008B73E00083C
:1000D000B73E0008C314000881140008551B00082F
:1000E000B73E0008B73E0008B73E0008B73E00081C
:1000F000B73E0008B73E0008B73E0008B73E00080C
:10010000B73E0008B73E0008B73E0008B73E0008FB
:10011000B73E0008B73E0008B73E0008B73E0008EB
:10012000B73E0008B73E0008B73E0008B73E0008DB
:1001300000F002F800F03AF80AA090E8000C8244BF
:100140008344AAF10107DA4501D100F02FF8AFF29C
:10015000090EBAE80F0013F0010F18BFFB1A43F0A5
:10016000010318471C4000003C400000103A24BF27
:1001700078C878C1FAD8520724BF30C830C144BF0C
:1001800004680C607047000000230024002500264E
:10019000103A28BF78C1FBD8520728BF30C148BFEA
:1001A0000B6070471FB51FBD10B510BD03F089FF70
:1001B0001146FFF7F7FF00F07BF803F0A7FF03B449
:1001C000FFF7F2FF03BC03F0AFFF000010B502F031
:1001D000F9FC4FF4803002F015FD102003F084FB91
:1001E000022003F06DFB002002F091FD002002F0E0
:1001F000A0FD4FF4806002F093FD4FF40021C81081
:1002000002F068FD012002F071FD00BF392002F00C
:100210001CFD0028FAD0022002F06BFD00BF02F0A6
:1002200071FD0828FBD101213D2002F039FE01219A
:10023000880302F035FE0121480402F03EFE012150
:10024000880402F03AFE0121480502F036FE10BD96
:1002500008B54FF4E06002F0C3FA27208DF80000E3
:1002600000208DF801008DF8020001208DF80300B8
:10027000684602F0BAFA26208DF8000000208DF8BA
:1002800001008DF8020001208DF80300684602F09D
:10029000ACFA25208DF8000000208DF801008DF8C3
:1002A000020001208DF80300684602F09EFA08BDA6
:1002B000FFF7CEFF03F081FE00F024F8FFF786FF82
:1002C00000F048FB0BA003F098F8182000F087FD21
:1002D00000F0C9FF01F07AFC01F099FC01F021FD6A
:1002E00001F0D1FD00F051F802E0012001F03DFEE7
:1002F000FBE7000053495354454D204143494C49C5
:10030000594F520030B516480068164AB0FBF2F15A
:10031000B1F1807F01D301201DE021F07F40401E1C
:100320004FF0E022506150170F22002807DA130720
:100330001D0E0D4B00F00F04241F1D5503E0130785
:100340001C0E0A4B1C5400BF00204FF0E0229061AD
:1003500007201061002008B100BFFEE730BD00009B
:10036000B800002040420F0018ED00E000E400E07B
:10037000002105E0002200E0521C8242FCDB491C07
:1003800040F2EE239942F5DB704700B585B00121BC
:100390008E4803F02AF98D4803F090F801214805B2
:1003A00002F08BFD0121082002F07AFDC020ADF89B
:1003B000100003208DF812001C208DF8130004A9F2
:1003C000834802F0B7FA0020ADF804004BF6FF7046
:1003D000ADF80600FE20ADF808004FF48060ADF8DF
:1003E0000A00FE20ADF80C004CF250300090694637
:1003F000764803F07CF801221102744803F060F99A
:1004000005B000BD2DE9F04704460E46924642F283
:100410001079254604F0FF082D12EFB201216B4838
:1004200003F007F900BF00BF6A49684803F0E2F92A
:100430000028F9D00022A021644803F050F942F2CC
:10044000107900BF6449614803F0D4F90028F9D05D
:1004500039465E4803F03DF942F2107900BF5E492B
:10046000891C5A4803F0C6F90028F8D0414657487D
:1004700003F02FF942F2107900BF5749891C534805
:1004800003F0B8F90028F8D03146504803F021F9BC
:1004900042F2107900BF5049891C4C4803F0AAF978
:1004A0000028F8D00121494803F0CFF80A20FFF7CF
:1004B0005FFFBDE8F0872DE9F04704468A4642F227
:1004C00010784FF000092546E7B22D12EEB2012157
:1004D0003E4803F0AEF800BF00BF3E493B4803F082
:1004E00089F90028F9D00022A021384803F0F7F854
:1004F00042F2107800BF3849344803F07BF90028F5
:10050000F9D03146314803F0E4F842F2107800BFE8
:100510003149891C2D4803F06DF90028F8D039467F
:100520002A4803F0D6F842F2107800BF2A49891C05
:10053000264803F05FF90028F8D00121234803F092
:1005400078F842F2107800BF2249204803F052F9AF
:100550000028F9D00122A1211C4803F0C0F842F282
:10056000107800BF1B49491C184803F043F90028C4
:10057000F8D00021154803F074F842F2107800BF5B
:1005800014493F31114803F035F90028F8D0012112
:100590000E4803F05AF80D4803F09DF88146BDE877
:1005A000F08701460A4610887047B0B532274FF0F1
:1005B000006500BF002405E0084801F05BFFAD1CAA
:1005C00004F10104B4F5806FF6DBB0BD00540040C7
:1005D000000C01400100030082000700A08601001A
:1005E0001FB54FF4165000900820ADF8040000200D
:1005F000ADF80600ADF80800ADF80C000C20ADF821
:100600000A006946FE4802F0F2FC0121FC4802F0B3
:100610007AFD012240F22551F94802F080FD1FBD0C
:1006200000B587B0002240F22551F64802F077FD70
:100630004FF4E13003900020ADF81000ADF8120047
:10064000ADF81400ADF818000C20ADF8160003A9A1
:10065000EC4802F0CCFC03A9EB4802F0C8FC0020F7
:10066000ADF80400ADF806004FF40070ADF80800D6
:100670000020ADF80A0001A9E24802F02DFD01A911
:10068000E14802F029FD012240F22551DD4802F047
:1006900046FD0121DB4802F036FD0121DA4802F077
:1006A00032FD07B000BD08B54FF48060ADF8000022
:1006B00018208DF8030003208DF802006946D34806
:1006C00002F038F94FF40060ADF8000004208DF816
:1006D00003006946CD4802F02DF908BD08B5042095
:1006E000ADF8000018208DF8030003208DF80200FB
:1006F0006946C74802F01EF90820ADF80000042042
:100700008DF803006946C24802F014F90220ADF8E2
:10071000000010208DF8030003208DF802006946C8
:10072000BB4802F007F908BD08B54FF40070ADF8FA
:10073000000018208DF8030003208DF802006946A0
:10074000B34802F0F7F84FF48060ADF800000420E1
:100750008DF803006946AE4802F0ECF808BD08B514
:100760000121AC4802F0B7F94FF48050ADF8000019
:1007700010208DF8030003208DF802006946A4487C
:1007800002F0D8F84FF44060ADF8000010208DF86A
:10079000030003208DF8020069469F4802F0CAF862
:1007A0004FF40040ADF8000010208DF80300032046
:1007B0008DF802006946964802F0BCF84FF40041FB
:1007C000934802F066F94FF44061934802F061F9F2
:1007D00008BD00B585B00121080302F061FB0020CF
:1007E000ADF800004FF48270ADF802000020ADF8C3
:1007F00004000220ADF806000120ADF80800400218
:10080000ADF80A003820ADF80C000020ADF80E005D
:100810000720ADF810006946804801F081FE0121F3
:100820007E4801F022FF05B000BD08B5012104207B
:1008300002F036FBE020ADF8000003208DF8020046
:1008400018208DF803006946714802F073F81020F3
:10085000ADF800008DF8030003208DF80200694612
:100860006D4802F067F810216B4802F010F9202063
:10087000ADF8000010208DF8030003208DF8020071
:100880006946654802F056F82021634802F0FFF8F7
:1008900008BD08B54EF20F00ADF8000010208DF82D
:1008A000030003208DF8020069465B4802F042F81D
:1008B00042F20300ADF8000010208DF80300032081
:1008C0008DF802006946524802F034F84FF49870EF
:1008D000ADF8000010208DF8030003208DF8020011
:1008E00069464A4802F026F84EF20F014A4802F0E3
:1008F000D0F80121464802F0CCF808BD08B54FF405
:100900006040ADF8000004208DF8030003208DF84E
:10091000020069463D4802F00DF84FF47070ADF8E2
:10092000000004208DF8030003208DF802006946C2
:10093000394801F0FFFF4FF48070ADF8000004204B
:100940008DF8030003208DF802006946304801F05D
:10095000F1FF08BD10B5FFF7D1FFFFF79AFFFFF7D2
:1009600064FFFFF736FFFFF7FAFEFFF7DDFEFFF744
:10097000B5FEFFF798FEFFF753FEFFF731FE10BDFF
:1009800000B587B0002240F225511E4802F0C7FB97
:100990004FF4165003900020ADF81000ADF812008F
:1009A000ADF81400ADF818000C20ADF8160003A93E
:1009B000144802F01CFB03A9134802F018FB0020A6
:1009C000ADF80400ADF806004FF40070ADF8080073
:1009D0000020ADF80A0001A90A4802F07DFB01A938
:1009E000094802F079FB012240F22551054802F046
:1009F00096FB0121034802F086FB012102480FE02B
:100A0000004400400038014000480040000C014014
:100A10000008014000023000001001400030014099
:100A200002F071FB07B000BD08B540F20740ADF819
:100A3000000010208DF8030003208DF802006946A5
:100A40009D4801F077FF40F207419B4802F021F8F2
:100A500008BD08B50820ADF8000004208DF803009B
:100A600003208DF802006946934801F063FF0420DB
:100A7000ADF800008DF8030003208DF802006946F0
:100A80008E4801F057FF4FF48050ADF8000004206D
:100A90008DF8030003208DF802006946884801F0B4
:100AA00049FF0821844801F0F4FF0421834801F044
:100AB000F0FF4FF48051824801F0EBFF08BD00B514
:100AC00085B00121480502F0F8F90121082002F063
:100AD000E7F9C020ADF8000003208DF802001C20CB
:100AE0008DF803006946744801F024FF754802F050
:100AF000E5FC0020ADF808004BF6FF70ADF80A00E9
:100B00003020ADF80C004FF48060ADF80E0000010D
:100B1000ADF810006C48019001216A4802F065FDB3
:100B200001A9684802F0E3FC0121082002F0B8F9AD
:100B30000121480502F0C1F905B000BD08B5032048
:100B4000ADF8000010208DF8030003208DF802009E
:100B500069465E4801F0EEFE03215C4801F099FF12
:100B600008BD00B587B00121080302F099F9E02023
:100B7000ADF8040001208DF8060018208DF807005C
:100B800001A9524801F0D6FE3020ADF80400012042
:100B90008DF8060010208DF8070001A9484801F0E3
:100BA000C9FE1021464801F072FF0020ADF8080090
:100BB0004FF48270ADF80A000020ADF80C00ADF8DB
:100BC0000E00ADF810004FF40070ADF812001020C8
:100BD000ADF814000020ADF816000720ADF818009D
:100BE00002A93B4801F09CFC0121394801F03DFD80
:100BF00007B000BD00B587B00121880302F05DF9A0
:100C00004FF46040ADF8040003208DF80600182072
:100C10008DF8070001A9284801F08CFE4020ADF8AE
:100C2000040003208DF8060010208DF8070001A9AC
:100C3000234801F07FFE4FF48050ADF804000320FC
:100C40008DF8060010208DF8070001A91A4801F060
:100C500071FE4020ADF8040003208DF8060004204A
:100C60008DF8070001A9164801F064FE0020ADF8D8
:100C700008004FF48270ADF80A000020ADF80C00B7
:100C8000ADF80E00ADF810004FF40070ADF8120092
:100C90000820ADF814000020ADF816000720ADF8CC
:100CA000180002A90B4801F03BFC0121094801F0A2
:100CB000DCFC07B000BD0000000C01400014014046
:100CC0000010014000540040801A06000008014056
:100CD000003001400038004010B504464FF4805108
:100CE000FE4801F0D4FE00E0641E012CFCDB4FF452
:100CF0008051FA4801F0CDFE10BD10B54FF480616F
:100D0000F74801F0C4FE502001F0B4FB4FF48061BD
:100D1000F34801F0BEFE502001F0ACFB4FF48061BF
:100D2000EF4801F0B4FE10BD10B5002436E04FF4DA
:100D30000041EA4801F0ADFE4FF40061E84801F0DF
:100D4000A8FEE848007800F0010040B14FF40041EF
:100D5000E24801F09CFE0A2001F08CFB07E04FF412
:100D60000041DE4801F095FE0A2001F083FBDD48DA
:100D700000784010DB4908704FF40061D84801F05A
:100D800086FE0A2001F076FB4FF40061D44801F0A2
:100D900080FE0A2001F06EFB601CC4B2082CC6DB8A
:100DA00010BD10B5002415E0012C03D1CE48007809
:100DB000CC490870022C03D1CB480079C94908708E
:100DC000032C03D1C848007AC6490870FFF7ACFF6E
:100DD000601CC4B2042CE7DBFFF78FFF10BD10B519
:100DE0000446012C07D1C048806840F08000BE490D
:100DF0008860FFF7D6FF022C07D1BB48806840F01F
:100E00004000B9498860FFF7CCFF032C07D1B648F2
:100E1000806840F02000B4498860FFF7C2FF042CCE
:100E200007D1B148806840F01000AF498860FFF7F3
:100E3000B8FF052C07D1AC48806840F00800AA49EB
:100E40008860FFF7AEFF062C07D1A748806840F006
:100E50000400A5498860FFF7A4FF072C07D1A2482A
:100E6000806840F00200A0498860FFF79AFF082CD4
:100E700007D19D48806840F001009B498860FFF7DA
:100E800090FF092C07D19848406840F080009649AF
:100E90004860FFF786FF0A2C07D19348406840F06E
:100EA000400091494860FFF77CFF0B2C07D18E482A
:100EB000406840F020008C494860FFF772FF0C2C1E
:100EC00007D18948406840F0100087494860FFF723
:100ED00068FF0D2C07D18448406840F00800824923
:100EE0004860FFF75EFF0E2C07D17F48406840F056
:100EF00004007D494860FFF754FF0F2C07D17A4862
:100F0000406840F0020078494860FFF74AFF102C23
:100F100007D17548406840F0010073494860FFF709
:100F200040FF112C07D17048006840F080006E49E6
:100F30000860FFF736FF122C07D16B48006840F0BD
:100F4000400069490860FFF72CFF132C07D1664861
:100F5000006840F0200064490860FFF722FF142C6D
:100F600007D16148006840F010005F490860FFF752
:100F700018FF152C07D15C48006840F008005A495A
:100F80000860FFF70EFF162C07D15748006840F0A5
:100F9000040055490860FFF704FF172C07D1524899
:100FA000006840F0020050490860FFF7FAFE182C74
:100FB00007D14D48006840F001004B490860FFF739
:100FC000F0FE10BD10B50446012C07D14648007A4A
:100FD00000F07F0044498860FFF7E3FE022C07D150
:100FE0004148007A00F0BF003F498860FFF7D9FE12
:100FF000032C07D13C48007A00F0DF003A498860B2
:10100000FFF7CFFE042C07D13748007A00F0EF003D
:1010100035498860FFF7C5FE052C07D13248007AB4
:1010200000F0F70030498860FFF7BBFE062C07D1BF
:101030002D48007A00F0FB002B498860FFF7B1FED5
:10104000072C07D12848007A00F0FD002649886067
:10105000FFF7A7FE082C07D12348007A00F0FE0016
:1010600021498860FFF79DFE092C07D11E480079B1
:1010700000F07F001C494860FFF793FE0A2C07D15F
:101080001948007900F0BF0017494860FFF789FE52
:101090000B2C07D11448007900F0DF00124948609A
:1010A000FFF77FFE0C2C07D10F48007900F0EF000E
:1010B0000D494860FFF775FE0D2C07D10A480079ED
:1010C00000F0F70008494860FFF76BFE0E2C10D1C6
:1010D0000548007900F0FB00034907E000080140E3
:1010E000001001407B000020CC0000204860FFF78A
:1010F00058FE0F2C07D1DF48007900F0FD00DD49D4
:101100004860FFF74EFE102C07D1DA48007900F056
:10111000FE00D8494860FFF744FE112C07D1D5489E
:10112000007800F07F00D3490860FFF73AFE122CE8
:1011300007D1D048007800F0BF00CE490860FFF723
:1011400030FE132C07D1CB48007800F0DF00C949EE
:101150000860FFF726FE142C07D1C648007800F07F
:10116000EF00C4490860FFF71CFE152C07D1C148E9
:10117000007800F0F700BF490860FFF712FE162C58
:1011800007D1BC48007800F0FB00BA490860FFF7BF
:1011900008FE172C07D1B748007800F0FD00B549CC
:1011A0000860FFF7FEFD182C07D1B248007800F068
:1011B000FE00B0490860FFF7F4FD10BD10B504460D
:1011C00024B94FF48051AC4801F063FC012C03D1E9
:1011D0002103A94801F05BFC022C0BD11720FFF77B
:1011E000FEFDE002FFF778FD1720FFF7EBFEE002BF
:1011F000FFF772FD032C11D14FF480519E4801F08E
:1012000046FC4FF48050FFF767FD4FF480519A4839
:1012100001F03FFC4FF48050FFF75EFD042C11D12C
:101220001520FFF7DCFD1620FFF7D9FDA002FFF720
:1012300053FD1520FFF7C6FE1620FFF7C3FEA002E0
:10124000FFF74AFD052C0DD11620FFF7C8FD4FF41E
:101250008050FFF741FD1620FFF7B4FE4FF4805099
:10126000FFF73AFD10BD10B5002420E01120FFF774
:10127000B6FD1220FFF7A6FE1320FFF7A3FE1420F1
:10128000FFF7ADFD44F6206001F0F4F81120FFF700
:1012900099FE1220FFF7A3FD1320FFF7A0FD1420F5
:1012A000FFF790FE44F6206001F0E4F8641C052C82
:1012B000DCDB1220FFF786FE1320FFF783FE10BD54
:1012C00070B504465CB91120FFF77CFE1220FFF7D1
:1012D00079FE1320FFF776FE1420FFF773FE012C32
:1012E0000BD11120FFF77BFD1220FFF76BFE1320BF
:1012F000FFF768FE1420FFF765FE032C0BD11120C9
:10130000FFF760FE1220FFF76AFD1320FFF75AFE79
:101310001420FFF757FE052C0BD11120FFF752FECA
:101320001220FFF74FFE1320FFF759FD1420FFF79F
:1013300049FE072C0BD11120FFF744FE1220FFF7C6
:1013400041FE1320FFF73EFE1420FFF748FD022C5C
:1013500001D1012000E00020042C01D1012100E096
:1013600000210843062C01D1012100E0002108439F
:10137000082C01D1012100E00021084370B30025B1
:1013800028E01120FFF71EFE1220FFF71BFE13209E
:10139000FFF718FE1420FFF715FE42F2107001F05F
:1013A00069F8022C02D11120FFF719FD042C02D19B
:1013B0001220FFF714FD062C02D11320FFF70FFDBA
:1013C000082C02D11420FFF70AFD4FF4FA6001F057
:1013D00051F86D1C322DD4DBFEF76AFF70BD70B57D
:1013E0000446012C24D100251EE01120FFF7F7FC54
:1013F0001220FFF7F4FC1320FFF7F1FC1420FFF795
:10140000EEFC1E4801F036F81420FFF7DBFD132038
:10141000FFF7D8FD1220FFF7D5FD1120FFF7D2FD11
:10142000164801F027F86D1C142DDEDBFEF740FF97
:10143000022C1DD11120FFF7D2FC1220FFF7CFFCA8
:101440001320FFF7CCFC1420FFF7C9FC0B4801F078
:1014500011F81420FFF7B6FD1320FFF7B3FD12209B
:10146000FFF7B0FD1120FFF7ADFD044801F002F8D1
:1014700070BD0000CC00002000080140605B03004C
:1014800010B540F22551FE4801F02EFFC0B10221F7
:10149000FC4801F0FEFA40F22551F94801F04EFFF8
:1014A000F74801F0A1FEF849087008460078F749AE
:1014B000F74A12788854F6480078401CF4490870BE
:1014C00010BD2DE9F04100240027002540F22551F0
:1014D000F04801F009FF00287ED040F22551ED4888
:1014E00001F02CFFEB4801F07FFEEB490870084645
:1014F0000078EA49EA4A12788854E9480078401CA2
:10150000E7490870E4480178E64801F069FE00BF49
:101510008021E04801F0D2FE0028F9D0E0480078B0
:10152000B0F5FA7F02DB0020DD490870DE48007864
:10153000012812D1D94800784E280ED1D7484079D9
:101540004C280AD1D548C079502806D1D348407BD1
:10155000442802D10220D4490870D44800780128D8
:101560000AD1CE4800784F2806D1CC4840784B2885
:1015700002D10220CD490870CC48007802280AD157
:10158000C64800784F2806D1C44840784B2802D17D
:101590000320C6490870C6480078012820D1BF48FA
:1015A000407843281CD1BD488078532818D1BB48C7
:1015B000C0784D2814D1B9480079492810D1B748CE
:1015C00040794E280CD1B5488079532808D1B348CA
:1015D000C07A312804D100E0BAE20220B449087090
:1015E000B4480078012819D1AC4800782B2815D1CF
:1015F000AA484078432811D1A848807852280DD1B4
:10160000A648C078452809D1A448407A312805D198
:101610000220A84908700020A7490870A548007852
:10162000012816D19D4800782B2812D19B4840787C
:1016300043280ED19948807852280AD19748C0781B
:10164000452806D19548407A302802D101209A4990
:1016500008709848007802281ED1904800784328E6
:101660001AD18E4840784F2816D18C4880784E2861
:1016700012D18A48407A47280ED18848807A50286B
:101680000AD18648C07A522806D18448007B532864
:1016900002D10320874908708648007803282AD1A0
:1016A0007E4800782B2826D17C484078532822D1C8
:1016B0007A48807841281ED17848C07850281AD1BD
:1016C00076484079522816D1744880793A2812D148
:1016D0007248C07920280ED17048007A31280AD18A
:1016E0006E48407A2C2806D16C48807A312802D185
:1016F0000420704908707148007801280AD16748B1
:1017000000784F2806D1654840784B2802D1022046
:101710006A4908706948007803280AD15F48007850
:101720004F2806D15D4840784B2802D104206349F8
:1017300008706248007805285AD1584840784828EF
:1017400056D15648C078542852D15448407941283F
:101750004ED15248C07954284AD15048807A4E28F8
:1017600046D14E48807C2C2842D14C48C07B322840
:101770000BD14A48007C302807D14848407C3028AB
:1017800003D100204D49087032E04448007D0D2807
:1017900005D14248407D0A2801D1012000E0002007
:1017A0003E49497D0D2905D13C49897D0A2901D150
:1017B000012100E0002108433849897D0D2905D128
:1017C0003649C97D0A2901D1012100E000210843E1
:1017D0003249C97D0D2905D13049097E0A2901D137
:1017E000012100E00021084310B1082033490870AE
:1017F0002A48407843282BD12848C078452827D14B
:101800002648C079522823D12448807A3A281FD10B
:101810002248007B53281BD12048407B492817D100
:101820001E48807B4D2813D11C48807C74280FD122
:101830001A48C07D65280BD1002603E00020174917
:101840008855761C142EF9DB0620FFF739FD00BF02
:1018500012484078432848D110488078502844D115
:101860000E48C078492840D10C4800794E283CD118
:101870000A48C0794E2838D10848007A4F281FE01E
:1018800000440040000801408C000020CE020020EF
:101890007E000020003801407C000020D80000209D
:1018A0007D00002000480040800000207F000020D4
:1018B00088000020810000208B0000208200002092
:1018C00013D1B548407A54280FD1B348807C4428BE
:1018D0000BD1002603E00020AF498855761C142E5A
:1018E000F9DB0620FFF7ECFC00BFAC4800780128CC
:1018F0000AD1A94800784F2806D1A74840784B283C
:1019000002D10220A5490870A448007803285AD1C2
:10191000A1484078482856D19F48C078542852D1D1
:101920009D48407941284ED19B48C07954284AD1DE
:101930009948807A4E2846D19748807C2C2842D1FD
:101940009548C07B32280BD19348007C302807D1C2
:101950009148407C302803D104209049087032E03F
:101960008D48007D0D2805D18B48407D0A2801D186
:10197000012000E000208849497D0D2905D18649D4
:10198000897D0A2901D1012100E000210843824913
:10199000897D0D2905D18049C97D0A2901D10121FF
:1019A00000E0002108437C49C97D0D2905D17A4911
:1019B000097E0A2901D1012100E00021084310B16C
:1019C00008207649087075480078052801D1012063
:1019D00000E00020704909782B2901D1012100E0A5
:1019E0000021084010B36C48407848281ED16A484E
:1019F000807854281AD16848C078542816D166488F
:101A00000079502812D16448407952280ED162489A
:101A1000807945280AD16048C079412806D15E48BE
:101A2000007A442802D106205C4908705B4800789F
:101A3000062801D1012000E00020574909784F29EC
:101A400001D1012100E00021084030B15248407826
:101A50004B2802D1072051490870504800780728C8
:101A600016D1002412E04C48005D44280DD1002519
:101A7000A71C00BF05E04848C05D494948556D1C9A
:101A80007F1C04F1FC008542F5DB641C142CEADBAE
:101A900044480078801E4049085C0D2858D14148D0
:101AA0000078401E085C0A2852D13E48007802287F
:101AB0004EDB00203CE03849095C2B2937D1364AFF
:101AC000411C515C432932D1811C515C53292ED1D8
:101AD000C11C515C51292AD100F10801515C302907
:101AE00001D1012100E000212B4B00F109029A5C99
:101AF000302A01D1012200E000221143B9B1264A67
:101B0000C11D515C2C2908D13021274A1170224A6D
:101B1000811D515C244A517009E01F4A811D515CAE
:101B2000214A11701C4AC11D515C1F4A5170401C52
:101B30001E28C0DB00221B490978891E164B5A5407
:101B400018490978491E5A540021164A117000BFDD
:101B5000BDE8F08170477047704711E013A001F0B5
:101B60004CFC00BF1748006800F4E06016490843C9
:101B7000001D14490860BFF34F8F00BF00BFFEE790
:101B8000ECE700BFFEE700BFFEE700BFFEE77047DF
:101B90007047704770470000D80000208A0000207E
:101BA000D20100207D0000208400002020444F4E00
:101BB000414E494D204B494C49544C454E44490DEA
:101BC0000A0000000CED00E00000FA0510B501204D
:101BD000FFF776FB4FF48071F74800F05AFFF7A04B
:101BE00001F00BFC0520FFF7E9FAF74800F042FC92
:101BF0004FF48071F04800F04AFFF4A001F0FDFBC3
:101C00000520FFF7DBFAF44800F034FC10BD10B5F6
:101C10000320FFF755FB0120F049087029E0F0A0F0
:101C200001F0A6FBF0A001F0E8FB0520FFF7C6FAE3
:101C3000F4480078401CF3490870084600783228C0
:101C400017DD0320FFF73CFBEFA001F0D6FB0020DF
:101C5000EC49087000BFF148006800F4E060F0490A
:101C60000843001DED490860BFF34F8F00BF00BF60
:101C7000FEE7DA4800780128D1D0EAA001F0BDFBE8
:101C8000EDA001F075FB47F2305000F0F3FB0520AA
:101C9000FFF794FAEBA001F06BFB47F2305000F035
:101CA000E9FB0520FFF78AFAE9A001F061FB47F2A2
:101CB000305000F0DFFB0520FFF780FAE6A001F0CE
:101CC00057FB47F2305000F0D5FB0520FFF776FABE
:101CD0000120E44908700520FFF7F2FAE2A001F0C4
:101CE00047FB47F2305000F0C5FB0520FFF766FACE
:101CF00012E00520FFF762FAC2480078401CC14993
:101D0000087008460078322806DD0020087006209A
:101D1000FFF7D6FAFEF7CCFAD24800780128E8D0CF
:101D200010BD10B50520FFF749FA0720FFF7C8FAE4
:101D30000120D1490870AAA001F01AFBA24800F0C6
:101D400099FBC3A001F014FB9F4800F093FB22E035
:101D50000520FFF733FAC9A001F00AFBCA4800F0DA
:101D600089FBCAA001F049FBC74800F083FBA548E6
:101D70000078401CA34908700846007832280ADD24
:101D8000C7A001F03AFB00209E4908700820FFF729
:101D900097FAFEF78DFAB84800780128D8D00020CD
:101DA00098490870C3A001F028FB0420FFF706FA49
:101DB000C3A001F022FBC9A001F0DAFA47F23050CB
:101DC00000F058FBCDA001F0D3FA47F2305000F0FC
:101DD00051FB0520FFF7F2F9D0A001F0C9FA47F254
:101DE000305000F047FB19E0D0A001F0C1FA47F2F3
:101DF000305000F03FFB0520FFF7E0F98148007804
:101E0000401C8049087008460078322806DD002012
:101E100008700820FFF754FAFEF74AFA964800784F
:101E20000228E1D000207749087021E0C3A001F02A
:101E30009FFAC64800F01EFB0520FFF7BFF9714866
:101E40000078401C6F490870C1A001F0D6FA6D48B7
:101E5000007832280CDDC1A001F0CFFA0820FFF78E
:101E60002FFA00208449087066490870FEF720FAAE
:101E7000814800780328D9D0002062490870BAA0B0
:101E800001F0BBFA10BD10B5BEA001F071FA47F227
:101E9000305000F0EFFA0520FFF790F9BCA001F0F8
:101EA00067FA47F2305000F0E5FA0520FFF786F9AF
:101EB000BA48007830280FD1B848407830280BD184
:101EC0001120FEF78CFF1220FFF77CF81320FFF79C
:101ED00079F81420FFF776F8B048007830280FD151
:101EE000AE48407839280BDC1120FEF778FF12202D
:101EF000FEF775FF1320FFF765F81420FFF762F86F
:101F0000A648007831280FD1A448407839280BDC46
:101F10001120FEF764FF1220FEF761FF1320FEF789
:101F20005EFF1420FFF74EF89C480078322801D15C
:101F3000012000E0002099490978332901D10121CD
:101F400000E00021084358B11120FEF748FF12209D
:101F5000FEF745FF1320FEF742FF1420FEF73FFF78
:101F600000208E490870487010BD04460420FFF719
:101F700025F98BA001F02AFA134800F07BFA012022
:101F8000904908700420FFF719F98FA001F0F0F9CB
:101F90003D4800F06FFA012C05D18F4801F0E8F9B7
:101FA0000A2000F067FA384800F064FA2CE10420B7
:101FB000FFF704F912E10000000C0140204D4F53DF
:101FC0004645545F4F464600905F0100204D4F53F9
:101FD0004645545F4F4E0000A0BB0D007F0000201F
:101FE00041540D0A000000004154204B4F4D555400
:101FF000204345564142492042454B4C454E4959A4
:102000004F5200008E0000204154204B4F4D55543C
:102010002043455641424920594F4B000CED00E00A
:102020000000FA054154204F4B2043455641424998
:102030002047454C4449000041542B434D47463D01
:10204000310D0A0041542B434D45453D320D0A00E8
:10205000415456310D0A000041542B435344543D22
:10206000310D0A008800002041542B43534D494E46
:10207000533F0D0A000000008100002041542B4313
:102080005245473F0D0A0000A086010020475052EC
:10209000535F42454B4C454E49594F52000000009A
:1020A0002047505253204241474C414E414D4144FC
:1020B0004900000020475052535F4F4B0000000082
:1020C000204E4554574F524B20415941524C41529A
:1020D0004920594150494C49594F520041542B53C2
:1020E000415042523D332C312C22434F4E545950D3
:1020F00045222C2247505253220D0A0041542B53A3
:10210000415042523D332C312C2241504E222C2240
:10211000696E7465726E6574220D0A0041542B530A
:10212000415042523D312C310D0A000041542B5395
:10213000415042523D342C310D0A000041542B5382
:10214000415042523D322C310D0A0000D0FB0100BB
:1021500020495020414C44490000000020495020B3
:10216000414C414D41444900204E4554574F524B3C
:1021700020415941524C41524920594150494C4407
:102180004900000041542B474D520D0A0000000049
:1021900041542B4353510D0A0000000084000020DD
:1021A00020534552564552204241474C414E4959D1
:1021B0004F522056455249204F4B554E4143414BBB
:1021C0000D0A00008A00002041542B485454504905
:1021D0004E49540D0A0000003841000853A001F098
:1021E0000CF95B4800F046F95A480078401C594900
:1021F000087008460078322806DD0020087056A0D6
:1022000001F0FBF8FEF754F85948007801283FF434
:10221000CEAE00204F49087056A001F0EEF84C48B1
:1022200000F028F903205249087058A001F0A0F8E6
:10223000474800F01FF922E00420FEF7BFFF58A036
:1022400001F0DBF8424800F015F942480078401CE4
:102250004049087046480078082804D100204449C5
:102260000870FEF725F83B480078322807DD00208B
:102270003849087054A001F0C0F8FEF719F83C483E
:1022800000780328D8D000203249087055A001F00A
:10229000B4F82F4800F0EEF805203549087059A031
:1022A00001F066F82A4800F0E5F818E00420FEF78F
:1022B00085FF58A001F0A1F8254800F0DBF825487B
:1022C0000078401C2349087008460078322806DD53
:1022D0000020087056A001F090F8FDF7E9FF2448AF
:1022E00000780528E2D000201A49087054A001F0B7
:1022F00084F8174800F0BEF856A001F07EF81448A4
:1023000000F0B8F800BF0520194908703DA001F0A1
:102310002FF80F4800F0AEF802E00420FEF74EFF61
:10232000134800780528F8D0EDE70000204F4B5502
:102330004D41204144524553204345564142492096
:1023400042454B4C454E49594F520D0A0000000082
:10235000A08601008E000020204F4B554D412041AA
:10236000445245532020484154410D0A00000000CA
:102370008A000020204F4B554D4120414452455387
:10238000204241534152494C490D0A0041542B48C7
:10239000545450414354494F4E3D300D0A00000003
:1023A000204F4B554D412041445245532054414DFF
:1023B000414D204345564142492042454B4C454EF4
:1023C00049594F520D0A0000204F4B554D412041B5
:1023D000445245532054414D414D20484154410DF4
:1023E0000A000000204F4B554D41204144524553B7
:1023F0002054414D414D204241534152494C490DD9
:102400000A00000041542B48545450524541440D99
:102410000A000000204F4B554D4120434556414294
:10242000492042454B4C454E49594F520D0A000038
:10243000204F4B554D412020484154410D0A00008A
:10244000204F4B554D41204241534152494C490D7B
:102450000A000000204F4B554E414E20444154414C
:102460004C41520D0A000000002000E0401C0A28E8
:10247000FCDB704710B504462046E11704EB917170
:102480008910114A11601148046017E00F48006874
:10249000401E0E490860FFF7E7FF0C4800680A4934
:1024A0000968884205DD4FF48051094800F0F1FACF
:1024B00004E04FF48051064800F0E9FA0348006850
:1024C0000028E3DA10BD0000A00000209C000020DE
:1024D0000008014010B50446BE48844208D10121DD
:1024E000801400F0F7FC0021A01400F0F3FC16E0CB
:1024F000B948844208D10121001400F0F8FC002101
:10250000201400F0F4FC0AE0B448844207D1012111
:10251000C01300F0ECFC0021E01300F0E8FC10BD5B
:1025200010B50022028802F441520B884C882343E4
:102530008C882343CC8823430C8923434C89234331
:102540008C892343CC8923431A430280838B4FF227
:10255000FF74234083830B8A038210BD2DE9F04F63
:1025600085B005460C464FF0000902274FF00008E1
:102570004FF0010B0026B246A88B4FF240010840F5
:10258000A88302202884B5F81C90A068022801D1F5
:1025900000BF38E0A08810B94FF0010B01E04FF008
:1025A000020B8D48854200D100E000BF684600F074
:1025B0000AFCDDF800A0E088B0F5007F0AD14FEA00
:1025C0001A2000EB80004000A168B0FBF1F0401D34
:1025D00086B20BE04FEA4B10BAFBF0F000EB800044
:1025E0004000A168B0FBF1F0401D86B20A20B6FBA6
:1025F000F0F606F00108A6EB0800C0F34F074FF60F
:10260000FF7000EA0828022F01DBFF2F02DD0227FE
:102610004FF00008E08840EA080038432884A0888A
:10262000A1890843618808432188084340F4006079
:1026300040EA0909A5F81C9005B0BDE8F08F00211B
:10264000018041808180C180018141818181C1817E
:102650000721018270470021018041808180C18073
:102660000221816000218181704721B1028842F0FE
:102670004002028004E002884FF6BF731A400280D5
:10268000704721B1828B42F48062828304E0828BA6
:102690004FF6FF331A408283704730B50024002381
:1026A0000C110125A540ABB21AB185881D43858068
:1026B00002E085889D43858030BD1AB183880B4335
:1026C000838002E083888B438380704781817047D9
:1026D0000146888970474FF6FF62914204D0028814
:1026E00042F48072028004E002884FF6FF631A40D1
:1026F0000280704721B1828842F00402828004E0A7
:1027000082884FF6FB731A408280704702884FF22E
:10271000FF731A40028002880A43028070470188D2
:1027200041F480510180704721B1028842F4005287
:10273000028004E002884DF6FF731A400280704761
:1027400002460020012901D0108B00E0908A7047DA
:102750000146088A7047B1F5804F04D1028842F4DF
:102760008042028004E002884BF6FF731A40028028
:1027700070470246002013890B400BB1012000E096
:1027800000207047CA4302817047F0B5024600201E
:1027900000240023002501F00F070126BE40B4B23B
:1027A0000B1101269E40B3B2968806EA03051689EE
:1027B000264016B10DB1012000E00020F0BD10B59B
:1027C000002201F00F040123A3409AB2D3430381F6
:1027D00010BD00000030014000380040003C0040C7
:1027E00031490143314A1160704770B5002100231F
:1027F0000F22C47804B32D4C246804F4E064C4F5BB
:10280000E064210AC1F10403CA40447804FA03F1E8
:102810008478144021430901254C0678A155047899
:1028200004F01F050124AC4005786D11AD0005F1E1
:10283000E025C5F8004109E0047804F01F050124F3
:10284000AC401C4D0678761145F8264070BD1A4AFA
:102850000A400243154B1B1F1A60704739B1134AD7
:10286000121D12680243114B1B1D1A6006E00F4A2D
:10287000121D126882430D4B1B1D1A6070470428FD
:1028800008D14FF0E021096941F004014FF0E02246
:10289000116107E04FF0E021096921F004014FF0D8
:1028A000E0221161704700000000FA050CED00E025
:1028B00000E400E080E100E080FFFF1F10B5044667
:1028C000BA48844208D10121042000F003FB002112
:1028D000042000F0FFFA22E0B548844208D101212B
:1028E000082000F0F7FA0021082000F0F3FA16E0C3
:1028F000B048844208D10121102000F0EBFA0021F9
:10290000102000F0E7FA0AE0AB48844207D1012129
:10291000202000F0DFFA0021202000F0DBFA10BDBB
:1029200010B50121084600F0D5FA0021012000F081
:10293000D1FA10BD2DE9F041024600250026002005
:1029400000230024002791F803C00CF00F0591F834
:1029500003C00CF0100CBCF1000F03D091F802C0C2
:102960004CEA050591F800C0BCF1000F31D01468A5
:1029700000202BE04FF0010C0CFA00F3B1F800C07E
:102980000CEA03069E4220D183004FF00F0C0CFA94
:1029900003F7BC4305FA03FC4CEA040491F803C0B6
:1029A000BCF1280F06D14FF0010C0CFA00FCC2F864
:1029B00014C00AE091F803C0BCF1480F05D14FF0F4
:1029C000010C0CFA00FCC2F810C0401C0828D1D33E
:1029D0001460B1F800C0BCF1FF0F34DD5468002072
:1029E0002EE000F1080C4FF0010808FA0CF3B1F8E2
:1029F00000C00CEA03069E4221D183004FF00F0C69
:102A00000CFA03F7BC4305FA03FC4CEA040491F802
:102A100003C0BCF1280F05D100F1080C08FA0CF82E
:102A2000C2F8148091F803C0BCF1480F07D100F13F
:102A3000080C4FF0010808FA0CF8C2F81080401C8E
:102A40000828CED35460BDE8F0814FF6FF710180B5
:102A5000022181700421C1707047024600209368F2
:102A60000B400BB1012000E0002070470146886850
:102A700080B2704702460020D3680B400BB10120A2
:102A800000E0002070470146C86880B270470161CD
:102A90007047416170470AB1016100E041617047D0
:102AA000C16070474FF480320A4382618161826164
:102AB00082698269704702460020404B18684FF6D1
:102AC0008073184040EA021008433C4B186070477E
:102AD0003B49C8617047F0B50A4600230024002135
:102AE000002500F00046B6F1004F02D1334EF169E7
:102AF00001E0324E7168C0F3034583B200F4401622
:102B0000B6F5401F08D121F070612C4E766826F092
:102B100070662A4F7E6012E000F48016B6F5801FC2
:102B200006D1032606FA05F4A14341F0706106E0E0
:102B3000460D360103FA06F6B14341F0706122B149
:102B4000460D360103FA06F6314300F00046B6F1B1
:102B5000004F02D1194EF16101E0184E7160F0BDD5
:102B600030B500228B071C0F0F2303FA04F2134B1E
:102B700008338C1053F824309343104C08348D10D4
:102B800044F8253023468C1053F824308C07240F4A
:102B900000FA04F42343094C08348D1044F825301E
:102BA00030BD0749DC310860704700000008014073
:102BB000000C0140001001400014014000000140E1
:102BC00000002042DF48006840F00100DD49086055
:102BD00008464068DC490840DA4948600846006811
:102BE000DA490840D74908600846006820F4802088
:102BF00008600846406820F4FE0048604FF41F005B
:102C000088607047CF49096821F48031CD4A11604E
:102C10001146096821F480211160B0F5803F03D08E
:102C2000B0F5802F0ED106E0C649096841F4803125
:102C3000C44A116007E0C349096841F4A021C14AB0
:102C4000116000E000BF00BF704710B501460022D0
:102C5000002300204A11012A02D1BA4C236806E061
:102C6000022A02D1B74C236A01E0B64C636A01F034
:102C70001F02012494401C400CB1012000E0002000
:102C800010BD38B5002000900024002500BF312081
:102C9000FFF7DBFF05460098401C00900098B0F558
:102CA000A06F01D0002DF2D03120FFF7CEFF08B188
:102CB000012400E00024204638BD01460020A14A3E
:102CC000106820F0F80040EAC10010607047A04989
:102CD00008607047024600209A4B586820F47C1028
:102CE00042EA01031843974B5860704798490866B9
:102CF000704701460020934A506820F003000843C3
:102D0000506070478F48406800F00C0070470146E3
:102D100000208C4A506820F0F00008435060704753
:102D200001460020874A506820F4E0600843506064
:102D3000704701460020834A506820F4605040EA02
:102D4000C1005060704729B17E4A527A02437D4BE0
:102D50005A7204E07B4A527A82437A4B5A72704725
:102D60007B49D8310860704701460020754A506899
:102D700020F440400843506070470021714A2032DF
:102D80001170704A82F82010012802D004280AD15C
:102D900004E001216B4A2032117005E00521694AE7
:102DA0002032117000E000BF00BF70476949086021
:102DB00070476449096A0143624A11627047654974
:102DC00044390860704730B50021002200240023F8
:102DD0005C4D6D6805F00C0121B1042905D008296E
:102DE00023D105E05C4D056022E05B4D05601FE0EE
:102DF000544D6D6805F47012524D6D6805F48034C1
:102E0000022505EB92421CB9544D554305600BE079
:102E10004C4D6D6805F400351DB1504D55430560AE
:102E200002E04D4D5543056002E04B4D056000BF8B
:102E300000BF444D6D6805F0F0010909484D6B5C19
:102E40000568DD4045603F4D6D6805F4E061090AA5
:102E5000434D6B5C4568DD4085603A4D6D6805F417
:102E60006051C90A3E4D6B5C4568DD40C560354D1B
:102E70006D6805F44041890B3A4D6B5CC568B5FB44
:102E8000F3F5056130BD29B12E4A526902432D4B3D
:102E90005A6104E02B4A526982432A4B5A617047B7
:102EA00029B1284A92690243264B9A6104E0254AD7
:102EB00092698243234B9A61704729B1214AD269B2
:102EC0000243204BDA6104E01E4AD26982431D4B63
:102ED000DA61704729B11B4AD2680243194BDA60A4
:102EE00004E0184AD2688243164BDA60704729B171
:102EF000144A12690243134B1A6104E0114A126921
:102F00008243104B1A61704712494039086070477C
:102F10000F49C86470470B49C87170470948406A37
:102F200040F0807007494862704701460020054A1A
:102F300092680A400AB1012000E000207047014970
:102F400088727047001002400000FFF8FFFFF6FE95
:102F5000000042428004424200127A0000093D0013
:102F6000A4000020B400002010B50446FB488442B1
:102F700009D101218803FFF7ADFF00214FF4804004
:102F8000FFF7A8FF32E0F648844209D10121480446
:102F9000FFF7ADFF00214FF40030FFF7A8FF25E059
:102FA000F048844209D101218804FFF7A0FF0021E5
:102FB0004FF48020FFF79BFF18E0EB48844209D1D3
:102FC0000121C804FFF793FF00214FF40020FFF711
:102FD0008EFF0BE0E548844208D101210805FFF788
:102FE00086FF00214FF48010FFF781FF10BD2DE90F
:102FF000F04786B005460E460024A24600BFA14613
:103000000027B08900B100BF2F462C8A4CF6FF7014
:103010000440F08804432C82AC894EF6F31004403F
:10302000B08831890843718908430443AC81AC8A74
:103030004FF6FF400440B0890443AC8201A8FFF77B
:10304000C2FEC648874202D1DDF810A001E0DDF8DB
:103050000CA0A88900F4004040B10AEBCA0000EBC4
:103060000A1031684900B0FBF1F807E00AEBCA002A
:1030700000EB0A1031688900B0FBF1F86420B8FB5E
:10308000F0F004012009642101FB1089A88900F4F3
:10309000004040B1322000EBC900B0FBF1F000F07D
:1030A0000700044308E0322000EB09106421B0FB64
:1030B000F1F000F00F0004432C8106B0BDE8F0876A
:1030C0004FF41651016000218180C18001810C21E3
:1030D000418100218181704710B502460020108A8D
:1030E0004FF2FF0318400B884C8823438C882343FE
:1030F000CC8823431843108210BD002101804180F9
:103100008180C180704721B1828942F4005282815E
:1031100004E082894DF6FF731A4082817047F0B552
:103120000346002400260025002040F66A17B94215
:1031300000D100BF1846C1F3421401F01F06012759
:1031400007FA06F5012C01D10C3004E0022C01D164
:10315000103000E014301AB107682F43076002E016
:103160000768AF430760F0BD1AB1838A0B438382BF
:1031700002E0838A8B4383827047028A4FF6F073A2
:103180001A400282028A0A430282704782894FF201
:10319000FF731A40828182890A438281704721B17C
:1031A000828942F00202828104E082894FF6FD7337
:1031B0001A4082817047028A4FF6DF731A400282FA
:1031C000028A0A430282704721B1028A42F4804295
:1031D000028204E0028A4BF6FF731A4002827047B3
:1031E000C1F308028280704701468888C0F3080056
:1031F0007047818941F0010181817047028BD2B211
:103200000283028B42EA012202837047028B02F49E
:103210007F420283028B0A430283704721B1828A74
:1032200042F02002828204E0828A4FF6DF731A4065
:103230008282704721B1828A42F01002828204E0C9
:10324000828A4FF6EF731A408282704721B1828AD8
:1032500042F00802828204E0828A4FF6F7731A4035
:103260008282704721B1828942F40042828103E068
:103270008289C2F30E028281704721B1828A42F4B0
:103280000062828204E0828A4FF2FF731A408282D7
:103290007047828A4FF6FB731A408282828A0A4301
:1032A0008282704721B1828A42F00202828204E067
:1032B000828A4FF6FD731A408282704702460020D0
:1032C000B1F5007F00D100BF13880B400BB1012086
:1032D00000E00020704701F40072B2F5007F00D1D9
:1032E00000BFCA430280704770B502460024002325
:1032F0000025002040F66A16B14200D100BFC1F39C
:10330000421501F01F03012606FA03F3012D02D135
:103310009689334006E0022D02D1168A334001E03F
:10332000968A33400C12012606FA04F416883440BB
:1033300013B10CB1012000E0002070BD10B50022D7
:10334000002340F66A14A14200D100BF0A120124F2
:103350009440A3B2DC43048010BD0000003801405B
:103360000044004000480040004C00400050004035
:1033700030B5044600250DE0605781B24B48FFF799
:103380002FFF00BF40214948FFF798FF0028F9D0E0
:10339000681C45B2605D0028EED1002530BD30B517
:1033A000044600250DE0605781B24148FFF718FF41
:1033B00000BF40213E48FFF781FF0028F9D0681C7C
:1033C00045B2605D0028EED1002530BD30B5044621
:1033D00000250DE0605781B23648FFF701FF00BFBE
:1033E00040213448FFF76AFF0028F9D0681C45B235
:1033F000605D0028EED1002530BD30B504460025C3
:103400002D48007840B30DE0605781B22948FFF79E
:10341000E7FE00BF40212748FFF750FF0028F9D002
:10342000681C45B2605D0028EED100250D212148C1
:10343000FFF7D6FE00BF40211E48FFF73FFF0028E0
:10344000F9D00A211B48FFF7CBFE00BF40211948E5
:10345000FFF734FF0028F9D030BD10B5044600BF97
:1034600040211448FFF72AFF0028F9D021461148CF
:10347000FFF7B6FE10BD10B5044600BF40210B4853
:10348000FFF71CFF0028F9D021460848FFF7A8FEE7
:1034900010BD10B5044606E0207800B904E014F829
:1034A000010BFFF7DAFFF7E700BF10BD003801405E
:1034B00000440040004800401200002010B50446BF
:1034C000F748844209D101214805FFF710FD00218A
:1034D0004FF40010FFF70BFD08E001218805FFF70E
:1034E00006FD00214FF48000FFF701FD10BD2DE91E
:1034F000F04385B004460D460026B1460427DFF8A8
:10350000A483A6884FF6C07006406846FFF75BFCB0
:10351000DDF80880E448B8FBF0F01FFA80F946EACD
:103520000906A68020884FF6FE71084020800026FC
:10353000DE49286888420CD828684000B8FBF0F0C3
:1035400087B2042F00DA04273E4309F101002084EA
:1035500027E0E8884BF6FF71884206D1286800EB27
:103560004000B8FBF0F087B209E0286800EBC0012A
:1035700001EB0010B8FBF0F087B247F48047C7F3C7
:103580000B0008B947F0010747F4004006434FF429
:10359000967009FB00F04FF47A7190FBF1F0401C3B
:1035A0002084A683208840F00100208026884FF6E2
:1035B000F5300640A8886989084306432680A88913
:1035C00029890843208105B0BDE8F08341F28831A4
:1035D0000160002181804BF6FF71C18000210181D3
:1035E00041814FF480418181704721B1028842F0CE
:1035F0000102028004E002884FF6FE731A40028046
:10360000704721B1828842F40062828004E082889F
:103610004FF2FF731A408280704721B1828842F4D2
:103620008052828004E082884EF6FF731A408280C6
:10363000704721B1028842F48072028004E002885F
:103640004FF6FF631A400280704721B1028842F4AE
:103650000072028004E002884FF6FF531A40028095
:10366000704721B1028842F48062028004E002883F
:103670004FF6FF331A40028070470A4600218189C5
:103680004FF60173194002F0FE0319438181704720
:1036900021B1828942F00102828104E082894FF6E1
:1036A000FE731A408281704721B1028842F04002C5
:1036B000028004E002884FF6BF731A400280704710
:1036C0001AB183880B43838002E083888B43838015
:1036D0007047018270470146088AC0B2704712B134
:1036E00041F0010102E04FF6FE731940018270477C
:1036F00008B502460020009000920098084400900F
:103700000098008808BD21B1028842F4004202807E
:1037100003E00288C2F30E0202807047B1F5006F29
:1037200004D1028842F40062028004E002884FF271
:10373000FF731A4002807047B1F5005F04D1028820
:1037400042F40052028004E002884DF6FF731A40F2
:103750000280704721B1028842F48052028004E066
:1037600002884EF6FF731A4002807047B1F5006F71
:1037700004D1028842F40062028004E002884FF221
:10378000FF731A400280704721B1028842F0200284
:10379000028004E002884FF6DF731A40028070470F
:1037A0000146088B0012704721B1028842F01002D6
:1037B000028004E002884FF6EF731A4002807047DF
:1037C00021B9028842F08002028004E002884FF6AC
:1037D0007F731A4002807047B1F5804F05D0828B0D
:1037E0004BF6FF731A40828303E0828B42F48042DF
:1037F0008283704770B50246002400250023002014
:10380000958A138B1B0445EA030626F07F4404EADD
:1038100001068E4201D1012000E0002070BD10B5EC
:1038200001460020002300228B8A0A8B120443EAFF
:10383000020424F07F4010BD0CB502460020002396
:103840000193009300920B0F019321F07F41019BA4
:103850001BB1009B1433009303E0090C009B183349
:103860000093009B1B680B400BB1012000E000207F
:103870000CBD002221F07F42D3438382704730B5D4
:10388000024600200023948801F0E06504EA154315
:1038900021F07F41948A0C4054B14BB1012008E0E3
:1038A0000054004000127A0040420F00A086010040
:1038B000002030BD002221F07F42D3438382704735
:1038C00001460020FE4A106800F0380008431060EE
:1038D0007047FB49096821F00801F94A1160114657
:1038E0000968014311607047F549096821F010012A
:1038F000F34A116011460968014311607047F148AD
:10390000EF494860F04848607047EE48EC4948602D
:10391000ED4848607047EA48006940F08000E84997
:1039200008617047E648006940F08000E44908619A
:1039300070470420E249C96801F0010109B1012082
:103940000EE0DF49C96801F0040109B1022007E077
:10395000DB49C96801F0100109B1032000E004202F
:10396000704700B502460423FFF7E3FF034603E078
:10397000FFF7DFFF0346521E012B01D1002AF7D1CA
:1039800002B90523184600BD30B5054604244FF49E
:103990003020FFF7E6FF0446042C19D1C84800691F
:1039A00040F00200C649086108464561006940F0E0
:1039B000400008614FF43020FFF7D3FF0446052C88
:1039C00006D0BF48006941F6FD710840BC49086156
:1039D000204630BD10B504244FF43020FFF7C1FF5E
:1039E0000446042C18D1B648006940F00400B449DC
:1039F00008610846006940F0400008614FF430203B
:103A0000FFF7AFFF0446052C06D0AD48006941F62C
:103A1000FB710840AA490861204610BD00B5024666
:103A20000423FFF786FF034603E0FFF782FF034608
:103A3000521E012B01D1002AF7D102B905231846E5
:103A400000BD10B504244FF43020FFF7E7FF044613
:103A5000042C18D19A48006940F004009849086184
:103A60000846006940F0400008614FF43020FFF73D
:103A7000D5FF0446052C06D09148006941F6FB713C
:103A800008408F490861204610BD00208C49C96953
:103A900001F0020109B1012000E00020704730B5BB
:103AA000A5250424FFF7F1FF00B100254FF43020D5
:103AB000FFF757FF0446042C3AD1824880498860BA
:103AC000814888600846006940F020000861084687
:103AD000006940F0400008614FF43020FFF741FFDB
:103AE0000446042C1BD17648006941F6DF7108407A
:103AF000734908610846006940F010000861734886
:103B00000580E002FFF72DFF0446052C10D06C481D
:103B1000006941F6EF7108406949086108E0052C29
:103B200006D06748006941F6EF71084064490861B2
:103B3000204630BD78B506460D460424002000908E
:103B4000E002FFF70EFF0446042C28D15C48006910
:103B500040F001005A4908613580E002FFF701FF9B
:103B60000446042C12D1B01C0090280C0099088047
:103B7000E002FFF7F6FE0446052C10D0504800691D
:103B800041F6FE7108404E49086108E0052C06D058
:103B90004B48006941F6FE710840494908612046DA
:103BA00078BD70B505460E460424E002FFF7D9FE45
:103BB0000446042C13D14248006940F001004049FA
:103BC00008612E80E002FFF7CCFE0446052C06D0EB
:103BD0003B48006941F6FE710840394908612046BA
:103BE00070BD70B505460E460424E002FFF7B9FE2D
:103BF0000446042C17D13348314988603248886024
:103C00000846006940F0100008612E80E002FFF7CE
:103C1000A8FE0446052C06D02948006941F6EF713C
:103C2000084027490861204670BD2DE9F04304464D
:103C30004FF6FF763746B046B1460425E443E6B278
:103C4000C4F30727C4F307484FEA1469E802FFF7F3
:103C500088FE0546042D4AD11A48194988601A4839
:103C600088600846006940F010000861FF2E06D009
:103C7000164808300680E802FFF773FE0546042D5B
:103C800008D1FF2F06D011480A300780E802FFF75D
:103C900068FE0546042D0AD1B8F1FF0F07D00B4886
:103CA0000C30A0F80080E802FFF75BFE0546042D0B
:103CB00014D1B9F1FF0F11D004480E3008E0000014
:103CC0000020024023016745AB89EFCD00F8FF1FBC
:103CD000A0F80090E802FFF744FE0546052D06D047
:103CE0006848006941F6EF71084066490861284656
:103CF000BDE8F08330B5054604244FF43020FFF7CB
:103D000030FE0446042C41D15F485E4988605F481C
:103D100088600846006940F0200008610846006994
:103D200040F0400008614FF43020FFF71AFE0446CF
:103D3000042C22D15348006941F6DF7108405149F3
:103D400008610846006940F0100008611DB10020BC
:103D50004F49088002E0A5204D4908804FF43020EB
:103D6000FFF7FFFD0446052C10D04648006941F6D8
:103D7000EF7108404349086108E0052C06D041482E
:103D8000006941F6DF7108403E490861204630BDB8
:103D9000F0B505460E46174604243B48394988606D
:103DA0003A488860E002FFF7DCFD0446042C19D194
:103DB0003448006940F010003249086147F0F800CB
:103DC000304328433249891C0880E002FFF7C9FDCF
:103DD0000446052C06D02B48006941F6EF710840D7
:103DE000284908612046F0BD2648C0698008704710
:103DF0002448006A704700202249096801F0200128
:103E000009B1012000E00020704729B11D4A126964
:103E100002431C4B1A6104E01A4A12698243194B8F
:103E20001A61704701460020012908D1154AD2695C
:103E300002F001020AB1012008E0002006E0114A68
:103E4000D2680A400AB1012000E0002070470D4905
:103E5000C860704704200B49C96801F0010109B12D
:103E600001200EE00749C96801F0040109B10220F0
:103E700007E00449C96801F0100109B1032000E01E
:103E8000042070470020024023016745AB89EFCD35
:103E900000F8FF1F70470B4880470B4981F30888E3
:103EA0000A480047FEE7FEE7FEE7FEE7FEE7FEE71B
:103EB000FEE7FEE7FEE7FEE705480649044A064B33
:103EC00070470000953E0008A00500203101000861
:103ED000A0030020A0050020A00300200CB50020B6
:103EE000019000906C48006840F480306A49086096
:103EF00000BF6948006800F4003000900198401C41
:103F00000190009818B90198B0F5A06FF1D16248FE
:103F1000006800F4003010B10120009001E00020A2
:103F200000900098012843D15C48006840F01000E0
:103F30005A4908600846006820F0030008600846F7
:103F4000006840F0020008605348406852494860E9
:103F50000846406848600846406840F48060486011
:103F60000846406820F47C1048600846406840F4E9
:103F7000E81048600846006840F08070086000BFA4
:103F80004548006800F000700028F9D042484068B9
:103F900020F00300404948600846406840F00200B5
:103FA000486000BF3C48406800F00C000828F9D188
:103FB0000CBD10B5FFF792FF10BD10B53648006874
:103FC00040F0010034490860084640683449084020
:103FD0003149486008460068324908402E49086067
:103FE0000846006820F4802008600846406820F4F5
:103FF000FE0048604FF41F008860FFF7DAFF4FF0C3
:1040000000602949086010BD10B500210020002281
:10401000214B5B6803F00C0121B1042906D008296B
:1040200028D107E0214B224C236027E01F4B204C76
:10403000236023E0184B5B6803F47010164B5B6839
:1040400003F48032022303EB904022B9194B43431F
:10405000174C23600DE0104B5B6803F4003323B171
:10406000144B4343124C236003E0104B4343104C6A
:10407000236003E00D4B0E4C236000BF00BF064BD6
:104080005B68C3F303130C4CE15C094B1B68CB402A
:10409000074C236010BD00000010024000200240C9
:1040A0000000FFF0FFFFF6FE08ED00E000127A00CE
:1040B000B800002000093D00BC0000207047704798
:1040C0007047754600F02CF8AE4605006946534629
:1040D00020F00700854618B020B5FFF7EDFEBDE8DB
:1040E00020404FF000064FF000074FF000084FF05F
:1040F000000B21F00701AC46ACE8C009ACE8C009F0
:10410000ACE8C009ACE8C0098D46704710B504465C
:10411000AFF300802046BDE81040FCF750B8000027
:10412000004870473C03002001491820ABBEFEE761
:10413000260002007047000041542B485454505050
:104140004152413D2255524C222C22687474703ADF
:104150002F2F7777772E6174626F746F6D6173792B
:104160006F6E2E636F6D2F736F6674776172652F3C
:1041700053575F56312E302E62696E220D0A0000B1
:10418000A041000800000020CC0000006C010008E5
:104190006C420008CC000020D40400008801000814
:1041A00039333535313030313335533031563031A4
:1041B00000000103393930303030303030303030A9
:1041C000303030303030303030300000000000000F
:1041D00000000000000000000000000000000000DF
:1041E00000000000000000000000000000000000CF
:1041F00000000000000000000000000000000000BF
:10420000000000000000000032000000000000007C
:10421000FF0F000800000000000000000000000088
:10422000000000000000000000000000000000008E
:10423000000000000000000000000000000000007E
:10424000000000000000000001020304010203045A
:10425000060708090204060800A24A04000000003C
:0C4260000000000001020304060708092A
:0400000508000131BD
:00000001FF
